S123F8008E00FF867FB710077F10098600B71035B610398A80B7103986F0B71030860297D5
S123F820A8FCFFB0DD9BFCFFB2DD9DBDF8C9CEFD24DF9F7F00837F00847F00857F0086BD1C
S123F840FBCDBDFB64B610008501275385022764BDF8E8BDF920BDF94ABDF9A79683BDFB47
S123F860A89684BDFBA89685BDFBA89686BDFBA8969BBDFBA8969CBDFBA8969DBDFBA8961F
S123F8809EBDFBA8BDFA32BDFAAEBDFB14BDFB93BDFA15BDF9F386809780BDFC7320A3DCA4
S123F8A085D399DD85DC832506D397DD8320A7C3000120F5DC859399DD85DC83250693975A
S123F8C0DD83209283000120F5B6100885102701397F009B7F009C7F009D7F009E7F00A820
S123F8E0B61008851027F939B61008851027013996A827148501260B7A00A8B610088510CF
S123F90027F9397C00A820F39683979B9684979C9685979D9686979E860197A8BDFD603902
S123F920B610088520270139DE9F080808088CFD4C2712DF9FEC00DD83EC02DD85B610085C
S123F940852027F939CEFD2820E996A885022616DC85D39DDDA42507DC83D39BDDA239DCC9
S123F96083C3000120F4DC831A939B25241A939B270FDC85939DDDA42510DC83939BDDA267
S123F98039DC851A939D250920E8DC8383000120EBDC9D9385DDA42507DC9B9383DDA239D8
S123F9A0DC9B83000120F4B610314497A681402422863F90A697A697A7270EDCA483035BA9
S123F9C0DDA425067A00A626F239DCA2830001DDA220F1804097A697A7270EDCA4C3035B63
S123F9E0DDA425067A00A626F239DCA2C30001DDA220F196A7C60A3DDD947F00927F009336
S123FA00BDFB1486CC9780BDFC739690BDFBA89691BDFBA83986C99780BDFC7396A88501E5
S123FA20260886209780BDFCA139865E9780BDFCA1397F00A1B6100484DFB7100486209761
S123FA408796A12654DC83DD88DC8805250CDD88B6100484BFB71004200ADD88B610048AEC
S123FA6040B710048A80B71004847FB710047A00879687811027068100270C20CC96A126FB
S123FA801CDC85DD8820C2B610048A10B7100484EFB7100496A1270939DCA220AADCA420A9
S123FAA0E27C00A1B610048A20B71004208FCC0000DD92DD94DC83DD8ADC85DD8CCEFD004E
S123FAC0DC8A1AA30022122742C6083A8CFD2826EF86C09780BDFC7339DC8CA3022518DDAB
S123FAE08CDC8AA300DD8ADC94E306DD942513DC92E304DD9220C9DD8CDC8A830001DD8A9D
S123FB0020DFDC92C30001DD9220E4DC8C1AA30224C720B5CE008E6F036F026F016F0086B2
S123FB20209796A6038D2AE703A6028D24E702A6018D1EE701A6008D18E700680769066935
S123FB4005690469036902690169007A009626D33916840F80052B02CB031784F080502B94
S123FB6002CB3039B6100085042712B6100085802716CC0001DD97CC4F8BDD9939CC000059
S123FB80DD97CC035BDD9939CC0083DD97CC126EDD9939968EBDFBA8968FBDFBA89690BD6A
S123FBA0FBA89691BDFBA839978284F0444444448D079682840F8D0139810922088B309735
S123FBC080BDFCA1398B379780BDFCA139BDFC27BDFC27BDFC27BDFC27BDFC278603BDFC00
S123FBE019BDFC278603BDFC19BDFC278603BDFC19BDFC278602BDFC19BDFC278628978093
S123FC00BDFC73860E9780BDFC7386019780BDFC7386069780BDFC7339B710038A40B710B0
S123FC2003843FB7100339CE01FF01010101010927037EFC2A398677B710078610B71003E9
S123FC408A40B71003B61003840826158610B710038A40B71003843FB71003867FB7100728
S123FC60398610B710038A40B71003843FB710037EFC3B9680840F9781968084F0444444FA
S123FC8044B710038A40B71003843FB710039681B710038A40B71003843FB71003BDFC3640
S123FCA0399680840F9781968084F0444444448A20B710038A40B71003843FB71003968100
S116FCC08A20B710038A40B71003843FB71003BDFC363970
S123FD00051EB852000F4240000D6CFB000028030000355A0000009F0000035B0000000AEC
S10BFD20000000560000000180
S123FD2809374BC711EB852023D70A3E33B645A347AE147C5C8216C86B851EBA7F6FD223C5
S107FD488F5C28F8A8
S11CFD60CEFD7918CE0000A60018A7000818088CFDC5270220F17E0000C9
S123FD79CEFFB0C60EF7103BE700C60FF7103B8D287F103BCEFFB018CE009B18A600C602D2
S123FD99F7103BA700C603F7103B8D0D7F103B081808188C009F26E3398606C6FF010101ED
S10EFDB95A270220F84A270220F139E3
S107FFB00000000049
S105FFFEF80005
S9030000FC
